:1000000000800010CD000000792D00007B2D000045
:100010007D2D00007F2D0000812D000000000000DC
:10002000000000000000000000000000832D000020
:10003000852D000000000000872D0000892D0000A4
:100040008B2D00008B2D00008B2D00008B2D0000D0
:100050008B2D0000051000008B2D00008B2D000063
:10006000191100008B2D00008B2D00008B2D00003E
:100070008B2D00008B2D00008B2D00008B2D0000A0
:100080008B2D00008B2D00008B2D00008B2D000090
:100090008B2D00008B2D00008B2D00008B2D000080
:1000A000CD2A00008B2D00008B2D00008B2D000031
:1000B0008B2D00008B2D00008B2D00008B2D000060
:1000C0008B2D00008B2D00008B2D000001488047F8
:1000D00001480047A92F00006532000040F21803D4
:1000E000C1F200031A780AB901201870704700BFE6
:1000F00040F20000C1F2000008B503682BB140F2E5
:100100000003C0F2000303B1984708BD08B54FF0E3
:10011000000000F007F908BD00B583B06B46184633
:1001200000F048FF009B002B21DD40F21003C1F2DC
:1001300000031B88002B1AD06B4640F23C00C1F232
:100140000000194600F064FE0346019340F21003DC
:10015000C1F200034FF000021A80019B4FF08200B1
:1001600040F23C01C1F200011A4602F045FC03B026
:1001700000BD00BF00B585B001AB184600F0BAF86D
:10018000019B002B18DD019B202BA8BF202303938C
:1001900003AB40F21C00C1F20000194600F042F827
:1001A0000346029302AB4FF0000040F21C01C1F283
:1001B00000011A4600F076FE05B000BD00B583B020
:1001C00000F04CFA0346ADF8063040F21A03C1F2D3
:1001D00000031B88BDF806209A4208D040F21A039B
:1001E000C1F20003BDF806201A8000F0D1FA03B076
:1001F00000BD00BF08B5FFF789FF02F099F94FF085
:10020000010002F00DFA40F28823C1F200031B78CE
:10021000002BF8D0FFF780FFFFF7D0FFFFF7AAFF12
:10022000F8E700BF84B001900091009B1B68029327
:10023000009B1B68029A9A42B8BF13460293029B26
:10024000039318E040F20C13C1F200035A6C02F061
:100250003F0140F20C13C1F20003595C019B19707D
:10026000019B03F10103019302F1010240F20C131F
:10027000C1F200035A64029B002B0CBF0023012330
:10028000DBB2029A02F1FF320292002BDAD1039B19
:10029000184604B0704700BF84B001900091009BE5
:1002A0001B680293029B03931CE040F20C13C1F203
:1002B00000031A6C02F03F01019B187840F20C1306
:1002C000C1F20003585402F1010240F20C13C1F2D2
:1002D00000031A64019B03F101030193029B03F1E4
:1002E000FF330293029B002BDFD1039B184604B01F
:1002F000704700BF82B0019040F20C13C1F20003BE
:100300001A6C40F20C13C1F200035B6CC3EB0203E6
:1003100003F03F02019B1A604FF00003184602B041
:10032000704700BF00B583B003468DF807309DF8D5
:100330000730002B1CD14FF0000000F0B9FA40F25A
:100340000803C1F20003186840F20803C1F2000379
:100350009B79194640F20803C1F200035B791A4603
:1003600040F20803C1F200031B7900F02DFB1BE0F3
:100370004FF0010000F09CFA40F20803C1F20003C4
:10038000186840F20803C1F200039B79194640F255
:100390000803C1F200035B791A4640F20803C1F278
:1003A00000031B7900F022FC40F21003C1F20003AD
:1003B0004FF001021A8000F051F903461A4640F24C
:1003C0007C03C1F200031A8040F20C13C1F2000357
:1003D0004FF000021A6440F20C13C1F200031A6CD1
:1003E00040F20C13C1F200035A6403B000BD00BF19
:1003F0004FF00103184670474FF00103184670474D
:1004000082B00346ADF806304FF00103184602B043
:10041000704700BF82B00346ADF806304FF00103CD
:10042000184602B0704700BF82B00346ADF80630F0
:100430004FF00103184602B0704700BF08B540F204
:100440007023C1F200031B781A4640F27023C1F2F8
:1004500000035B784FEA032342EA030240F2702371
:10046000C1F200039B784FEA034342EA030240F2E1
:100470007023C1F20003DB784FEA036342EA03030F
:100480001A4640F20803C1F200031A6040F27023DA
:10049000C1F200031A7940F20803C1F200031A7195
:1004A00040F27023C1F200035A7940F20803C1F20E
:1004B00000035A7140F27023C1F200039A7940F2AE
:1004C0000803C1F200039A714FF0000000F042FAF5
:1004D0004FF0000000F0ECF940F20803C1F2000315
:1004E000186840F20803C1F200039B79194640F2F4
:1004F0000803C1F200035B791A4640F20803C1F217
:1005000000031B7900F060FA4FF00103184608BDA4
:1005100040F20803C1F200031B68DAB240F2702314
:10052000C1F200031A7040F20803C1F200031B6815
:100530004FEA1323DAB240F27023C1F200035A707B
:1005400040F20803C1F200031B684FEA1343DAB21A
:1005500040F27023C1F200039A7040F20803C1F226
:1005600000031B684FEA1363DAB240F27023C1F252
:100570000003DA7040F20803C1F200031A7940F276
:100580007023C1F200031A7140F20803C1F20003A4
:100590005A7940F27023C1F200035A7140F2080305
:1005A000C1F200039A7940F27023C1F200039A71FC
:1005B0004FF001031846704782B00346ADF806308D
:1005C0004FF00103184602B0704700BF82B00346E7
:1005D000ADF806304FF00103184602B0704700BF77
:1005E00000B583B06B46184600F0E4FC6B4640F261
:1005F000CC00C1F20000194600F00AFC034601934A
:10060000019B002B0ADD019B4FF0820040F2CC01E0
:10061000C1F200011A4602F0EFF906E040F21003C1
:10062000C1F200034FF001021A8003B000BD00BF09
:1006300000B583B04FF0020040F28001C1F200012A
:1006400002F07EF90346019301AB40F28000C1F253
:1006500000001946FFF720FE03B000BD00B583B0CF
:1006600040F27C03C1F200034FF000021A800DF14A
:100670000603184600F0B4FCBDF806301BB2002B90
:100680000CDA40F27C03C1F200031B8843F0010343
:100690009AB240F27C03C1F200031A80BDF8063022
:1006A00003F40053002B0CD040F27C03C1F2000392
:1006B0001B8843F002039AB240F27C03C1F20003AC
:1006C0001A80BDF8063003F01003002B0CD040F266
:1006D0007C03C1F200031B8843F004039AB240F28A
:1006E0007C03C1F200031A80BDF8063003F4804396
:1006F000002B0CD040F27C03C1F200031B8843F0B6
:1007000008039AB240F27C03C1F200031A80BDF8DC
:10071000063003F00803002B0CD040F27C03C1F23A
:1007200000031B8843F010039AB240F27C03C1F22D
:1007300000031A80BDF8063003F00403002B0CD030
:1007400040F27C03C1F200031B8843F020039AB2FD
:1007500040F27C03C1F200031A80BDF8063003F0BA
:100760000203002B0CD040F27C03C1F200031B8873
:1007700043F040039AB240F27C03C1F200031A80B6
:1007800040F27C03C1F200031B88184603B000BD91
:1007900008B540F2C003C1F200036FF05E021A70A8
:1007A00040F2C003C1F200034FF020025A7040F241
:1007B000C003C1F200034FF000029A7040F2C00380
:1007C000C1F200034FF00002DA7040F2C003C1F240
:1007D00000034FF000021A7140F2C003C1F200039F
:1007E0004FF000025A7140F2C003C1F200034FF013
:1007F00002029A7140F2C003C1F200034FF00002FE
:10080000DA7140F27C03C1F200031B88DAB240F2D5
:10081000C003C1F200031A7240F27C03C1F200036C
:100820001B884FEA13239BB2DAB240F2C003C1F235
:1008300000035A724FF0810040F2C001C1F2000182
:100840004FF00A0202F0D8F808BD00BF82B003469C
:100850008DF807304EF20013CEF200039DF9072009
:100860004FEA52129DF8071001F01F014FF00100EE
:1008700000FA01F143F8221002B0704782B003463B
:100880008DF807304EF20013CEF200039DF90720D9
:100890004FEA52129DF8071001F01F014FF00100BE
:1008A00000FA01F102F1200243F8221002B0704771
:1008B00000B583B003468DF807309DF80730002B54
:1008C0001CD14FF00500FFF7D9FF4CF20003C4F232
:1008D00002034CF20002C4F20202126822F0F0029B
:1008E0001A604CF20003C4F202034CF20002C4F29C
:1008F0000202126842F050021A6029E04CF2000332
:10090000C4F20F034CF20002C4F20F02D2F8C4206A
:1009100042F00072C3F8C4204FF00800FFF7AEFFAA
:100920004CF20003C4F202034CF20002C4F20202D1
:10093000126822F00F021A604CF20003C4F20203A4
:100940004CF20002C4F20202126842F00A021A607B
:1009500003B000BD00B583B003468DF807309DF8A5
:100960000730002B17D14CF20003C4F202034CF203
:100970000002C4F20202126822F0F0021A604CF285
:100980000003C4F200034FF000025A604FF005006C
:10099000FFF774FF16E04CF20003C4F202034CF2BE
:1009A0000002C4F20202126822F00F021A604CF236
:1009B0000003C4F209034FF000025A604FF0080030
:1009C000FFF75CFF03B000BD00B589B00390029152
:1009D00001920093029B062B08D0072B0BD0052B0E
:1009E0000ED14FF000038DF813300DE04FF00103EE
:1009F0008DF8133008E04FF002038DF8133003E058
:100A00004FF003038DF81330009B03F1FF33012BEC
:100A100004D84FF004038DF8123003E04FF00003C8
:100A20008DF81230019B03F1FF33032B1ED801A276
:100A300052F823F0450A00004F0A0000590A00004E
:100A4000630A00004FF008038DF8113012E04FF0F8
:100A500018038DF811300DE04FF028038DF8113098
:100A600008E04FF038038DF8113003E04FF0000339
:100A70008DF8113040F2E413C1F200034FF0000290
:100A8000C3F8802040F2E413C1F20003D3F88020C1
:100A900040F2E413C1F20003C3F8842040F254137F
:100AA000C1F200034FF00002C3F8802040F254135B
:100AB000C1F20003D3F8802040F25413C1F20003C6
:100AC000C3F884204CF20003C4F20F03D3F8A8311A
:100AD0004FEA931303F003030693069B022B13D0F4
:100AE000032B1AD0012B08D040F21403C1F20003EB
:100AF0001B684FEA9303079317E040F21403C1F217
:100B000000031B68079310E040F21403C1F20003D6
:100B10001B684FEA5303079307E040F21403C1F246
:100B200000031B684FEAD3030793079B4FEA131296
:100B3000039BB2FBF3F305934CF20003C4F20003F2
:100B40004FF0000283F828204CF20003C4F20003A7
:100B50009DF813109DF8112041EA0202D1B29DF8D0
:100B6000122041EA0202D2B26FEA42626FEA526296
:100B7000D2B21A734CF20003C4F20003059AD2B247
:100B80001A704CF20003C4F20003059A4FEA1222D5
:100B9000D2B21A714CF20003C4F200039DF8131094
:100BA0009DF8112041EA0202D1B29DF8122041EADB
:100BB0000202D2B21A734CF20003C4F200034FF0E7
:100BC00003025A604CF20003C4F200034FF0070224
:100BD0001A7240F2DC13C1F200034FF001021A60F6
:100BE0004FF00500FFF732FE09B000BD00B589B037
:100BF0000390029101920093029B062B08D0072BD1
:100C00000BD0052B0ED14FF000038DF813300DE003
:100C10004FF001038DF8133008E04FF002038DF818
:100C2000133003E04FF003038DF81330009B03F102
:100C3000FF33012B04D84FF004038DF8123003E08A
:100C40004FF000038DF81230019B03F1FF33032BAB
:100C50001ED801A252F823F0690C0000730C0000AA
:100C60007D0C0000870C00004FF008038DF8113058
:100C700012E04FF018038DF811300DE04FF028030B
:100C80008DF8113008E04FF038038DF8113003E093
:100C90004FF000038DF8113040F2E413C1F200036D
:100CA0004FF00002C3F8802040F2E413C1F20003C9
:100CB000D3F8802040F2E413C1F20003C3F884208B
:100CC00040F25413C1F200034FF00002C3F8802039
:100CD00040F25413C1F20003D3F8802040F25413C1
:100CE000C1F20003C3F884204CF20003C4F20F03E6
:100CF000D3F8AC314FEA934303F003030693069B0A
:100D0000022B13D0032B1AD0012B08D040F214036E
:100D1000C1F200031B684FEA9303079317E040F208
:100D20001403C1F200031B68079310E040F21403A0
:100D3000C1F200031B684FEA5303079307E040F238
:100D40001403C1F200031B684FEAD3030793079B08
:100D50004FEA1312039BB2FBF3F305934CF200032B
:100D6000C4F209034FF0000283F828204CF200037C
:100D7000C4F209039DF813109DF8112041EA020204
:100D8000D1B29DF8122041EA0202D2B26FEA426269
:100D90006FEA5262D2B21A734CF20003C4F2090332
:100DA000059AD2B21A704CF20003C4F20903059AF4
:100DB0004FEA1222D2B21A714CF20003C4F20903B4
:100DC0009DF813109DF8112041EA0202D1B29DF85E
:100DD000122041EA0202D2B21A734CF20003C4F2AA
:100DE00009034FF003025A604CF20003C4F20903F6
:100DF0004FF007021A7240F2DC13C1F200034FF009
:100E000001021A604FF00800FFF720FD09B000BD95
:100E100084B001900091009B1B680293009B1B68AB
:100E2000029A9A42B8BF13460293029B039328E0AA
:100E300040F25413C1F20003D3F8842040F254135B
:100E4000C1F20003D3F880309A42F1D040F254133B
:100E5000C1F20003D3F8842002F07F0140F2541362
:100E6000C1F20003595C019B1970019B03F101035E
:100E7000019302F1010240F25413C1F20003C3F8DE
:100E80008420029B002B0CBF00230123DBB2029ABB
:100E900002F1FF320292002BCAD1039B184604B024
:100EA000704700BF86B00346029101928DF80F3063
:100EB000019B1B680493049B059340F2E413C1F269
:100EC0000003D3F8842040F2E413C1F20003D3F806
:100ED00080309A42F1D11EE040F2E413C1F20003E7
:100EE000D3F8802002F07F01029B187840F2E413CF
:100EF000C1F20003585402F1010240F2E413C1F2BE
:100F00000003C3F88020029B03F101030293049BBA
:100F100003F1FF330493049B002BDDD140F2DC137B
:100F2000C1F200031B68002B3FD040F2DC13C1F27A
:100F300000034FF000021A609DF80F30002B1AD109
:100F40004CF20003C4F2000340F2E412C1F20002CA
:100F5000D2F8841001F07F0040F2E412C1F20002E6
:100F6000125C1A7001F1010240F2E413C1F20003B5
:100F7000C3F8842019E04CF20003C4F2090340F2E4
:100F8000E412C1F20002D2F8841001F07F0040F2B6
:100F9000E412C1F20002125C1A7001F1010240F287
:100FA000E413C1F20003C3F88420059B184606B081
:100FB000704700BF82B0019040F25413C1F20003A9
:100FC000D3F8802040F25413C1F20003D3F88430E8
:100FD000C3EB020303F07F02019B1A6002B070476B
:100FE00082B0019040F2E013C1F200031A88019B25
:100FF0001A8040F2E013C1F200034FF000021A80A1
:1010000002B0704782B04CF20003C4F200039B6848
:101010000193019B03F00403002B21D1019B03F0FA
:101020000C03002B28D01CE040F25413C1F2000343
:10103000D3F8802002F07F014CF20003C4F20003D9
:101040001B78D8B240F25413C1F20003585402F195
:10105000010240F25413C1F20003C3F8802000E003
:1010600000BF4CF20003C4F200031B7DDBB203F0AF
:101070000103DBB2002BD7D1019B03F00203002B4D
:101080003AD040F2E413C1F20003D3F8802040F2DA
:10109000E413C1F20003D3F88430C3EB020303F07E
:1010A0007F03002B21D04CF20003C4F2000340F276
:1010B000E412C1F20002D2F8841001F07F0040F285
:1010C000E412C1F20002125C1A7001F1010240F256
:1010D000E413C1F20003C3F8842040F2DC13C1F230
:1010E00000034FF000021A6006E040F2DC13C1F288
:1010F00000034FF001021A604CF20003C4F2000337
:101100001B7DDBB21A4602F01E0240F2E013C1F270
:1011100000031A8002B0704782B04CF20003C4F2A0
:1011200009039B680193019B03F00403002B21D169
:10113000019B03F00C03002B28D01CE040F2541359
:10114000C1F20003D3F8802002F07F014CF20003CB
:10115000C4F209031B78D8B240F25413C1F2000361
:10116000585402F1010240F25413C1F20003C3F8D3
:10117000802000E000BF4CF20003C4F209031B7D95
:10118000DBB203F00103DBB2002BD7D1019B03F0EC
:101190000203002B3AD040F2E413C1F20003D3F86B
:1011A000802040F2E413C1F20003D3F88430C3EB93
:1011B000020303F07F03002B21D04CF20003C4F2A2
:1011C000090340F2E412C1F20002D2F8841001F0E7
:1011D0007F0040F2E412C1F20002125C1A7001F1C9
:1011E000010240F2E413C1F20003C3F8842040F28C
:1011F000DC13C1F200034FF000021A6006E040F277
:10120000DC13C1F200034FF001021A604CF200033C
:10121000C4F209031B7DDBB21A4602F01E0240F243
:10122000E013C1F200031A8002B0704740F2A0231D
:10123000C1F200034FF000021A8040F27C23C1F299
:1012400000034FF000021A7040F28823C1F200033D
:101250004FF000021A7040F27823C1F200034FF001
:1012600001121A6040F28423C1F200034FF0000221
:101270001A6040F28023C1F200034FF000021A60AE
:10128000704700BF08B54FF0000040F28C21C1F25A
:10129000000101F055FB08BD00B583B040F2982372
:1012A000C1F200039B88082B03D94FF00803019378
:1012B00005E040F29823C1F200039B88019340F2BD
:1012C0009823C1F200031B684FF080001946019A71
:1012D00001F092FB0346019340F29823C1F2000310
:1012E0001A68019B1A4440F29823C1F200031A6065
:1012F00040F29823C1F200039A88019B9BB2C3EB92
:1013000002039AB240F29823C1F200039A8003B01C
:1013100000BD00BF00B583B040F29823C1F20003C6
:101320001B684FF00000194601F00AFB03460193C9
:1013300040F29823C1F200031A68019B1A4440F25C
:101340009823C1F200031A6040F29823C1F200030F
:101350009A88019B9BB2C3EB02039AB240F2982396
:10136000C1F200039A8003B000BD00BF08B54FF082
:1013700080004FF000014FF0000201F03DFB08BD7E
:1013800008B54FF0000040F27021C1F2000101F0F9
:10139000D7FA08BD82B040F28C23C1F200031B785B
:1013A000C3F30403DBB2012B0ED0022B3AD0002B87
:1013B00040F0988040F2A022C1F2000240F298234F
:1013C000C1F200031A6090E040F28823C1F20003EA
:1013D0001B78002B23D040F28C23C1F200031A7932
:1013E00040F29423C1F200031B789A4217D240F2D4
:1013F0007023C1F200034FF000021A8040F2702304
:10140000C1F200034FF000021A8040F29823C1F2AB
:10141000000340F27022C1F200021A6065E04FF052
:10142000000364E040F28C23C1F200031B7903F057
:101430008F030093009B03F08003002B07D0009BD9
:1014400003F00F034FF4803202FA03F304E0009B31
:101450004FF0010202FA03F3019340F28823C1F234
:1014600000031B78002B04D1009B03F00F03002B1B
:1014700035D140F27823C1F200031A68019B02EAD9
:101480000303002B2BD040F27023C1F2000340F283
:101490008422C1F200021168019A01EA0202002AC4
:1014A0000CBF002201221A8040F27023C1F2000317
:1014B00040F28422C1F200021168019A01EA02029C
:1014C000002A0CBF002201221A8040F29823C1F2A8
:1014D000000340F27022C1F200021A6005E04FF0F2
:1014E000000304E04FF0000301E04FF00103184651
:1014F00002B0704700B585B0019040F28C23C1F274
:1015000000031B78C3F30403DBB2012B3AD0022B98
:101510003BD0002B40F0AB8040F28C23C1F20003A3
:101520005B88012B2BD1019B002B11D04FF00100C8
:1015300001F0F2F840F2A023C1F200031B8843F04F
:1015400002039AB240F2A023C1F200031A8091E094
:101550004FF0000001F0E0F840F2A023C1F20003D8
:101560001B881A464FF6FD73C0F2000302EA03031C
:101570001A4640F2A023C1F200031A807AE04FF02D
:10158000000379E04FF0000376E040F28C23C1F2D3
:1015900000031B7903F08F030293029B03F0800387
:1015A000002B07D0029B03F00F034FF4803202FAA6
:1015B00003F304E0029B4FF0010202FA03F30393EA
:1015C00040F28823C1F200031B78002B4CD0029B11
:1015D00003F00F03002B47D040F27823C1F2000341
:1015E0001A68039B02EA0303002B3DD040F28C23D0
:1015F000C1F200035B88002B33D1019B002B10D07C
:10160000029801F067F940F28423C1F200031A68DE
:10161000039B42EA030240F28423C1F200031A60F2
:1016200028E040F28023C1F200031A68039B02EA1B
:101630000303002B02D04FF001031DE0029801F0DC
:101640005FF9039B6FEA030240F28423C1F20003B7
:101650001B6802EA030240F28423C1F200031A600D
:1016600008E04FF0000307E04FF0000304E04FF004
:10167000000301E04FF00103184605B000BD00BFB4
:1016800040F28C23C1F200031B78C3F30403DBB2E6
:10169000002B11D140F28C23C1F200039B786FEA3A
:1016A00043636FEA5363DAB240F27C23C1F2000372
:1016B0001A704FF0010301E04FF000031846704725
:1016C00084B040F28C23C1F200031B78C3F30403FF
:1016D000DBB2002B03D0012B00F0968097E040F2A4
:1016E0008C23C1F20003DB78022B10D0032B4AD0ED
:1016F000012B7CD140F29823C1F2000343F2C422B3
:10170000C0F200021A604FF01203029372E043F23B
:10171000D823C0F2000301934FF00003039312E0BB
:10172000019B1B78002B0AD0019B9A78DB784FEA4B
:10173000032343EA02039BB2019A13440193039BE0
:1017400003F10103039340F28C23C1F200039B7861
:101750001A46039B9A42E3D1019B1B78002B02D1CE
:101760004FF000035FE040F29823C1F20003019ABA
:101770001A60019B9A78DB784FEA032343EA02035D
:101780009BB2029336E043F21C33C0F20003019394
:101790004FF0000303930CE0019B1B78002B04D057
:1017A000019B1B78019A13440193039B03F10103EE
:1017B000039340F28C23C1F200039B781A46039BEB
:1017C0009A42E9D1019B1B78002B02D14FF0000314
:1017D00029E040F29823C1F20003019A1A6040F216
:1017E0009823C1F200031B681B78029302E04FF0BC
:1017F000000318E040F29823C1F200039B881A46C8
:10180000029B9A4206D80CE04FF000030BE04FF029
:10181000000308E0029B9AB240F29823C1F2000351
:101820009A804FF00103184604B0704740F28C23B1
:10183000C1F200031B78C3F30403DBB2002B0BD10E
:1018400040F29823C1F2000340F28822C1F2000264
:101850001A604FF0010301E04FF000031846704793
:1018600000B587B04FF00003029340F28C23C1F221
:1018700000031B78C3F30403DBB2002B40F072813A
:1018800040F28C23C1F200039B78002B00F006810C
:1018900043F2D823C0F200030193F9E0019B5B7887
:1018A000042B00F0B680052B00F0B780022B40F02F
:1018B000E680019B5A7940F28C23C1F200039B78A9
:1018C0009A4240F0968040F28C23C1F200039A784D
:1018D00040F28823C1F200031A70019B1A7940F28A
:1018E0009423C1F200031A704FF0000303930BE03E
:1018F000039A40F26C23C1F200034FF000019954A7
:10190000039B03F101030393039B032BF0D94FF0D7
:10191000010303932AE0039B4FF0010202FA03F351
:101920001A4640F27823C1F200031B6802EA03035F
:10193000002B02D0039800F0A3FF039B4FF48032EA
:1019400002FA03F31A4640F27823C1F200031B683F
:1019500002EA0303002B05D0039B43F080031846E3
:1019600000F08EFF039B03F101030393039B0F2BF6
:10197000D1D940F27823C1F200034FF001121A606E
:1019800040F28423C1F200034FF000021A6040F2DB
:101990008023C1F200034FF000021A604FF00100F3
:1019A00000F0E0FE019BDB7903F04003002B0DD03B
:1019B00040F2A023C1F200031B8843F001039AB256
:1019C00040F2A023C1F200031A8058E040F2A023A5
:1019D000C1F200031B881A464FF6FE73C0F20003E3
:1019E00002EA03031A4640F2A023C1F200031A8060
:1019F00045E0019B0593019B9A78DB784FEA03232E
:101A000043EA02039BB2059A13440593059B019395
:101A10003EE0019BDB78029331E0029B002B2ED14C
:101A2000019B9B7803F08F030393039B03F08003D8
:101A3000002B07D0039B03F00F034FF4803202FA10
:101A400003F304E0039B4FF0010202FA03F3049353
:101A500040F27823C1F200031A68049B42EA0302B1
:101A600040F27823C1F200031A60019B184600F08F
:101A7000A9FE039800F0F0FE039800F017FF019B09
:101A80000593019B1B78059A13440593059B0193CD
:101A9000019B1B78002B7FF401AF51E040F28823BB
:101AA000C1F200034FF000021A704FF001030393DC
:101AB0002AE0039B4FF0010202FA03F31A4640F2B8
:101AC0007823C1F200031B6802EA0303002B02D053
:101AD000039800F0D5FE039B4FF4803202FA03F323
:101AE0001A4640F27823C1F200031B6802EA03039E
:101AF000002B05D0039B43F08003184600F0C0FE86
:101B0000039B03F101030393039B0F2BD1D940F2F5
:101B10007823C1F200034FF001121A6040F28423CF
:101B2000C1F200034FF000021A6040F28023C1F2BC
:101B300000034FF000021A604FF0000000F012FEA8
:101B400040F28C23C1F200039A7840F28823C1F25C
:101B500000031B789A4202D04FF0000304E04FF0DC
:101B6000010301E04FF00003184607B000BD00BFBD
:101B700040F28C23C1F200031B78C3F30403DBB2F1
:101B8000012B28D140F28823C1F200031B78002BDF
:101B90001ED040F28C23C1F200031A7940F2942344
:101BA000C1F200031B789A4212D240F28C23C1F298
:101BB00000031B791A4640F26C23C1F200031A4459
:101BC00040F29823C1F200031A604FF0010304E0D1
:101BD0004FF0000301E04FF000031846704700BFCC
:101BE00000B58BB04FF0000302934FF00003039356
:101BF0004FF0000304934FF00003059340F28C2351
:101C0000C1F200031B78C3F30403DBB2012B40F0E5
:101C1000FD8040F28823C1F200031B78002B02D123
:101C20004FF00003F4E04FF00003089343F2D82391
:101C3000C0F200030193E2E0019B5B78042B1ED00D
:101C4000052B4CD0022B40F0D180019B5A7940F2F9
:101C50008823C1F200031B789A4200F0C280019BE6
:101C60000993019B9A78DB784FEA032343EA020346
:101C70009BB2099A13440993099B0193BFE0019B0E
:101C80009B780293019BDB7803934FF0000305934D
:101C900040F28C23C1F200031B791A46029B9A4240
:101CA00040F0A18040F28C23C1F200039B781A46D9
:101CB000039B9A4240F099804FF001030893029AE7
:101CC00040F26C23C1F200039B5C0493029A039BD5
:101CD000D9B240F26C23C1F20003995486E040F27D
:101CE0008C23C1F200031B791A46029B9A427DD1D4
:101CF000019B9B7803F08F030693069B03F0800300
:101D0000002B07D0069B03F00F034FF4803202FA3A
:101D100003F304E0069B4FF0010202FA03F307937A
:101D200040F28C23C1F200039B781A46039B9A422F
:101D30002BD140F27823C1F200031A68079B42EAD4
:101D4000030240F27823C1F200031A60079B6FEA96
:101D5000030240F28423C1F200031B6802EA03027B
:101D600040F28423C1F200031A60019B184600F080
:101D700029FD069800F070FD069800F097FD059A81
:101D8000079B42EA0303059330E0039A049B9A42BF
:101D90002CD1059A079B02EA0303002B26D1079B4F
:101DA0006FEA030240F27823C1F200031B6802EAE3
:101DB000030240F27823C1F200031A60079B6FEA26
:101DC000030240F28423C1F200031B6802EA03020B
:101DD00040F28423C1F200031A60069800F050FD1F
:101DE00004E000BF02E000BF00E000BF019B0993D8
:101DF000019B1B78099A13440993099B0193019B4A
:101E00001B78002B7FF418AF089B01E04FF0000314
:101E100018460BB000BD00BF00B583B00190019B18
:101E200003F1FF33062B00F2988201A252F823F04F
:101E30004D1E000001220000E92200005B2300008B
:101E40005B2300003D23000047230000FFF71AFA40
:101E500040F28C23C1F200031B78C3F3C013DBB242
:101E6000184600F0F5FC40F28C23C1F20003DA883A
:101E700040F29823C1F200039A8040F28C23C1F211
:101E800000031B78C3F34113DBB2002B03D0012BFB
:101E900000F08880A7E140F28C23C1F200035B7858
:101EA0000B2B00F2798101A252F823F0DD1E000015
:101EB000EF1E000099210000051F0000992100007D
:101EC0001B1F00002D1F00003F1F0000571F0000B8
:101ED000691F00007F1F0000911F0000FFF75AFAE2
:101EE0000346002B00F05A81FFF7D6F959E04FF076
:101EF0000000FFF7FFFA0346002B00F05181FFF7C7
:101F000035FA4EE04FF00100FFF7F4FA0346002BDC
:101F100000F04881FFF72AFA43E0FFF7B1FB0346E0
:101F2000002B00F04181FFF721FA3AE0FFF7C8FBF0
:101F30000346002B00F03A81FFF7AEF931E04FF095
:101F4000000000F0C7FC40F29823C1F200034FF0FC
:101F500000029A8025E0FFF769FC0346002B00F0A1
:101F60002781FFF799F91CE0FFF77AFC0346002B65
:101F700000F02081FFF7FAF900F094FE11E0FFF77E
:101F8000F7FD0346002B00F01781FFF785F908E005
:101F9000FFF726FE0346002B00F01081FFF7E6F95D
:101FA00000BF2CE140F28C23C1F200031B78C3F385
:101FB0000403DBB2012B04D0022B00F00181002BC3
:101FC00011E140F28C23C1F200031B79002B07D0F2
:101FD00040F28C23C1F200031B79012B40F0F28008
:101FE00040F28C23C1F200035B78232B00F2EC80DB
:101FF00001A252F823F000BF892000009D200000BC
:10200000C1200000D520000005210000C9210000EA
:10201000C9210000C9210000C9210000C921000018
:10202000C9210000C9210000C9210000C921000008
:10203000C9210000C9210000C9210000C9210000F8
:10204000C9210000C9210000C9210000C9210000E8
:10205000C9210000C9210000C9210000C9210000D8
:10206000C9210000C9210000C9210000C9210000C8
:10207000C9210000C92100002321000037210000F0
:102080005B2100007921000040F29823C1F2000397
:1020900040F27022C1F200021A607CE0FEF7ACF957
:1020A0000346002B0BD040F29823C1F2000340F20C
:1020B0007022C1F200021A60FFF7EEF86BE069E0EF
:1020C00040F29823C1F2000340F27022C1F20002F4
:1020D0001A6060E040F28C23C1F200035B8818466E
:1020E000FEF798F90346002B0BD040F29823C1F27B
:1020F000000340F27022C1F200021A60FFF7CCF830
:1021000049E047E040F28C23C1F200035B881846A7
:10211000FEF78AF90346002B02D0FFF727F93AE0D1
:1021200038E040F29823C1F2000340F27022C1F27D
:1021300000021A602FE0FEF7EBF90346002B0BD0EC
:1021400040F29823C1F2000340F27022C1F2000273
:102150001A60FFF7A1F81EE01CE040F28C23C1F2E8
:1021600000035B881846FEF727FA0346002B02D0CF
:10217000FFF7FCF80FE00DE040F28C23C1F2000302
:102180005B881846FEF722FA0346002B1ED0FFF7A5
:10219000EDF800E027E032E000BF24E000BF22E0DD
:1021A00000BF20E000BF1EE000BF1CE000BF1AE03F
:1021B00000BF18E000BF16E000BF14E000BF12E04F
:1021C00000BF10E000BF0EE000BF0CE000BF0AE05F
:1021D00000BF08E000BF06E000BF04E000BF02E06F
:1021E00000BF00E000BF4FF0800000F073FB40F242
:1021F0009823C1F200034FF000029A80ADE0ACE0FA
:1022000040F28C23C1F200031B7803F08003002B03
:1022100067D140F29823C1F200039B88002B00F0A5
:102220009780FFF777F840F29823C1F200039B886C
:10223000002B40F08F8040F28C23C1F200031B780A
:10224000C3F34113DBB2002BC2D0012BC2D140F249
:102250008C23C1F200031B78C3F30403DBB2012B10
:1022600003D0022BB8D0002BBDE740F28C23C1F283
:1022700000031B79002B06D040F28C23C1F200032F
:102280001B79012BAAD140F28C23C1F200035B78A9
:10229000022B0CD0202B19D0002BA1D1FEF7A8F8CF
:1022A0000346002B02D0FFF761F818E016E040F279
:1022B0008C23C1F200035B881846FEF7A1F80346A1
:1022C000002B02D0FFF752F809E007E0FEF7B6F85E
:1022D0000346002B86D0FFF749F800E083E700BFF4
:1022E0003BE0FFF74DF838E040F28C23C1F20003E9
:1022F0001B7803F08003002B02D0FEF7CDFF2CE00B
:1023000040F27C23C1F200031B785BB2002B23DA7E
:1023100040F27C23C1F200031B781A4602F07F02D0
:1023200040F27C23C1F200031A7040F27C23C1F218
:1023300000031B78184600F0F3F90EE04FF00000A0
:1023400000F0DEFA09E04FF0800000F0D9FA04E076
:1023500000BF02E000BF00E000BF03B000BD00BF4F
:1023600082B003468DF807304EF20013CEF2000320
:102370009DF907204FEA52129DF8071001F01F0146
:102380004FF0010000FA01F143F8221002B070474B
:1023900084B00190019B03F00F034FEA43030393C2
:1023A000019B03F08003002B03D0039B03F1010387
:1023B0000393039B184604B0704700BF82B001909E
:1023C0004CF20003C5F200034FF01002C3F80822DC
:1023D0004CF20003C5F20003019AC3F810224CF23C
:1023E0000003C5F20003D3F8003203F01003002B02
:1023F000F5D002B0704700BF82B0019000914CF25E
:102400000003C5F200034FF01002C3F808224CF29B
:102410000003C5F20003019AC3F810224CF2000336
:10242000C5F20003D3F8003203F01003002BF5D0FF
:102430004CF20003C5F200034FF01002C3F808226B
:102440004CF20003C5F20003009AC3F810224CF2CC
:102450000003C5F20003D3F8003203F01003002B91
:10246000F5D002B0704700BF10B582B00190009166
:102470004CF20003C5F200034FF01002C3F808222B
:102480004CF20004C5F200040198FFF781FF0346F7
:102490004FEA034343F4A063C4F810324CF2000344
:1024A000C5F20003D3F8003203F01003002BF5D07F
:1024B0004CF20003C5F200034FF01002C3F80822EB
:1024C0004CF20003C5F20003009AC3F810224CF24C
:1024D0000003C5F20003D3F8003203F01003002B11
:1024E000F5D002B010BD00BF82B001904CF20003E5
:1024F000C5F200034FF03002C3F808224CF200038B
:10250000C5F20003019AC3F810224CF20003C5F291
:102510000003D3F8003203F02003002BF5D04CF277
:102520000003C5F20003D3F81432184602B0704716
:1025300008B54CF20003C4F202034CF20002C4F2EC
:102540000202526822F070525A604CF20003C4F248
:1025500002034CF20002C4F20202526842F0A0529E
:102560005A604CF20003C4F202034CF20002C4F2BF
:102570000202D26822F0405222F03002DA604CF2BD
:102580000003C4F202034CF20002C4F20202D26859
:1025900042F0005242F01002DA604CF20003C4F242
:1025A00002034CF20002C4F20202126922F4402239
:1025B0001A614CF20003C4F202034CF20002C4F2AE
:1025C0000202126942F480221A614CF20003C4F242
:1025D0000F034CF20002C4F20F02D2F8C42042F002
:1025E0000042C3F8C4204CF20003C5F200034FF0D0
:1025F0001A02C3F8F42F4CF20003C5F20003D3F81B
:10260000F83F03F01A031A2BF5D14FF01800FFF72B
:10261000A7FE00F01BF84FF0000000F081F808BDA5
:1026200000B583B00190019B002B04D040F2001351
:10263000C0F2010301E04FF4807340F20050C0F299
:10264000FE001946FFF7D8FE03B000BD4CF20003B0
:10265000C5F200034FF00002C3F848224CF2000319
:10266000C5F200034FF00802C3F84C224CF20003FD
:10267000C5F200034FF00102C3F848224CF20003F8
:10268000C5F200034FF00802C3F84C224CF20003DD
:10269000C5F20003D3F8003203F48073002BF5D0A9
:1026A0004CF20003C5F200034FF0FF32C3F83822AA
:1026B0004CF20003C5F200034FF0FF32C3F834229E
:1026C0004CF20003C5F200034FF0FF32C3F80822BA
:1026D0004CF20003C5F200034FF00C02C3F80422D1
:1026E000704700BF704700BF704700BF08B540F299
:1026F000A023C1F200031B8803F00203002B09D0C2
:1027000040F20050C0F2FE0040F20011C0F20101A0
:10271000FFF772FE08BD00BF82B0019002B07047A3
:1027200000B583B00190019B43F080034FEA03435F
:1027300043F4807340F20050C0F2D0001946FFF716
:102740005BFE019B43F080034FEA034343F4807335
:1027500040F20050C0F2D0001946FFF74DFE03B022
:1027600000BD00BF00B583B00190019B002B04D0D9
:1027700040F20013C0F2010301E04FF4807340F215
:102780000050C0F2D8001946FFF736FE4CF20003A5
:10279000C5F200034FF00302C3F844224CF20003D9
:1027A000C5F20003D3F8003203F48073002BF5D098
:1027B0004CF20003C5F200034FF48072C3F8082204
:1027C00003B000BD00B585B00190019B9B78184611
:1027D000FFF7DEFD034603934CF20003C5F200034E
:1027E0004CF20002C5F20002D2F84412039A4FF0F4
:1027F000010000FA02F241EA0202C3F844224CF25C
:102800000003C5F20003039AC3F848224CF2000308
:10281000C5F20003019A117952794FEA022242EA85
:10282000010292B2C3F84C224CF20003C5F200033D
:10283000D3F8003203F48073002BF5D04CF2000380
:10284000C5F200034FF48072C3F8082205B000BD42
:1028500082B0019002B0704700B583B0019001983A
:10286000FFF796FD03464FEA034343F4800343F426
:10287000A06318464FF48071FFF7BEFD03B000BDA2
:1028800000B583B001900198FFF782FD03464FEA3F
:10289000034343F4800343F4A063184640F200115D
:1028A000C0F22001FFF7A8FD03B000BD00B583B062
:1028B00001900198FFF76CFD03464FEA034343F490
:1028C000800343F4A06318464FF48071FFF794FD32
:1028D00003B000BD00B583B001900198FFF758FD2B
:1028E00003464FEA034343F4800343F4A0631846CE
:1028F00040F20011C0F20101FFF77EFD03B000BD00
:1029000000B583B001900198FFF742FD03464FEAFE
:10291000034343F4800343F4A06318464FF48071EB
:10292000FFF76AFD03B000BD00B583B001900198C8
:1029300040F20051C0F2F201FFF796FD03B000BD76
:1029400000B585B0019000914CF20003C5F2000380
:10295000019A02F00F024FEA820242F00102C3F82C
:1029600028224CF20003C5F20003D3F82032029370
:10297000029B03F40063002BF3D0029B4FEA8353C6
:102980004FEA935302934FF0000303930FE0009A32
:102990004CF20003C5F20003D3F818321360009B19
:1029A00003F104030093039B03F101030393029BD0
:1029B00003F103034FEA9302039B9A42E7D84CF2D8
:1029C0000003C5F200034FF00002C3F82822019B68
:1029D00041F2482242FA03F303F00103002B06D12F
:1029E000019840F20051C0F2F201FFF73DFD029B59
:1029F000184605B000BD00BF00B587B00390029136
:102A000001924CF20003C5F20003039A02F00F0298
:102A10004FEA820242F00202C3F828224CF200037D
:102A2000C5F20003019AC3F824224FF00003059376
:102A30000FE04CF20003C5F20003029A1268C3F8DB
:102A40001C22029B03F104030293059B03F1010383
:102A50000593019B03F103034FEA9302059B9A42FE
:102A6000E7D84CF20003C5F200034FF00002C3F8B0
:102A70002822039840F20051C0F2FA01FFF7F4FC5B
:102A8000019B184607B000BD00B583B040F200506E
:102A9000C0F2F500FFF792FC40F20020C0F2F50012
:102AA000FFF722FD0346019340F20020C0F2F5003B
:102AB000FFF71AFD03464FEA0323019A42EA030394
:102AC0000193019B184603B000BD00BF00B587B05D
:102AD0004CF20003C5F20003D3F800320093009BD0
:102AE00003F00803002B2FD04CF20003C5F20003C3
:102AF0004FF00802C3F8082240F20050C0F2FE0076
:102B0000FFF75CFC40F20020C0F2FE00FFF7ECFC97
:102B100003460193019B03F01003002B03D0FFF742
:102B200095FD00F0BBF8019B03F00803002B00F0BB
:102B3000B180019B03F00403002B02D0FFF7D2FD0C
:102B4000A9E0FFF7D1FDA6E0009B03F00403002BF2
:102B500000F0A1804FF0000305934CF20003C5F292
:102B60000003D3F8303204934FF00003029382E065
:102B7000049A059B9A4200F08380029B4FF0010269
:102B800002FA03F31A46049B02EA0303002B6ED0F9
:102B9000029B4FF0010202FA03F3059A42EA030393
:102BA0000593029B4FEA530303934CF20003C5F2D3
:102BB0000003029A4FF0010101FA02F2C3F8382231
:102BC0004CF20003C5F20003D3F8003203F02003F7
:102BD000002BF5D04CF20003C5F20003D3F81432F9
:102BE0000193029B03F00103002B2BD1029B002BCE
:102BF00014D1019B03F00403002B0FD043F2843364
:102C0000C0F200031B68002B08D043F28433C0F2EB
:102C100000031B684FF00100984728E0039A43F235
:102C20008433C0F2000353F82230002B1ED0039AE5
:102C300043F28433C0F2000353F822304FF0020015
:102C4000984714E0039A43F28433C0F2000353F828
:102C50002230002B0BD0039A43F28433C0F20003DE
:102C600053F822304FF00300984700E000BF029B6A
:102C700003F101030293029B1F2B7FF679AF00E063
:102C800000BF4CF20003C5F200034FF00402C3F88A
:102C9000082200E000BF07B000BD00BF08B5FEF786
:102CA000C5FA08BD704700BF00B585B00190019B13
:102CB000032B16D1FDF7D2FC0346ADF80E3040F2DF
:102CC0007E03C1F200031B88BDF80E209A4208D093
:102CD00040F27E03C1F20003BDF80E201A80FDF71A
:102CE00057FD05B000BD00BF00B583B00190019B4A
:102CF000022B02D0032B03D004E0FDF799FC01E086
:102D0000FDF76EFC03B000BD82B0019002B07047C9
:102D100082B0019002B0704782B0019002B070475B
:102D200082B0019002B0704782B0019002B070474B
:102D300082B0019002B0704782B0019002B070473B
:102D400082B0019002B0704782B0019002B070472B
:102D500082B0019002B0704782B0019002B070471B
:102D600082B0019002B0704782B0019002B070470B
:102D700082B001900091FEE7FEE7FEE7FEE7FEE786
:102D8000FEE7FEE7FEE7FEE7FEE7FEE74CF20003A4
:102D9000C4F20F03D3F888304FEA136303F0030340
:102DA000032B40F0AA804CF20003C4F20F03D3F8C7
:102DB0000C3103F00303032B00F2F48001A252F85C
:102DC00023F000BFD52D0000392E00009F2E0000FB
:102DD000D52D00004CF20003C4F20F03D3F8883065
:102DE0004FEA43434FEA534303F1010241F2002308
:102DF000C0F27A0303FB02F24CF20003C4F20F03A9
:102E0000D3F888304FEA134303F0FF0303F10103C3
:102E1000B2FBF3F24CF20003C4F20F03D3F8043117
:102E200003F0FF0303F10103B2FBF3F240F21403DA
:102E3000C1F200031A60B6E04CF20003C4F20F03C3
:102E4000D3F888304FEA43434FEA534303F101027A
:102E500043F20063C0F26E1303FB02F24CF2000374
:102E6000C4F20F03D3F888304FEA134303F0FF0393
:102E700003F10103B2FBF3F24CF20003C4F20F03BF
:102E8000D3F8043103F0FF0303F10103B2FBF3F2C3
:102E900040F21403C1F200031A6000BF83E04CF259
:102EA0000003C4F20F03D3F888304FEA43434FEADC
:102EB000534303F101034FEA03424CF20003C4F20F
:102EC0000F03D3F888304FEA134303F0FF0303F1F5
:102ED0000103B2FBF3F24CF20003C4F20F03D3F888
:102EE000043103F0FF0303F10103B2FBF3F240F2FC
:102EF0001403C1F200031A6055E04CF20003C4F25F
:102F00000F03D3F80C3103F00303032B4BD801A2BA
:102F100052F823F0252F0000512F00007D2F0000D4
:102F2000252F00004CF20003C4F20F03D3F8043144
:102F300003F0FF0303F1010240F60013C0F23D036A
:102F4000B3FBF2F240F21403C1F200031A602AE06C
:102F50004CF20003C4F20F03D3F8043103F0FF0373
:102F600003F1010241F60033C0F2B703B3FBF2F202
:102F700040F21403C1F200031A6014E04CF20003A3
:102F8000C4F20F03D3F8043103F0FF0303F101038C
:102F90004FF40042B2FBF3F240F21403C1F200031B
:102FA0001A6000E000BF70474CF20003C4F20F0348
:102FB0004FF02002C3F8A0214CF20003C4F20F032B
:102FC000D3F8A03103F02003002B09D04CF200030A
:102FD000C4F20F03D3F8A03103F04003002BF5D067
:102FE0004CF20003C4F20F034FF00302C3F80421B4
:102FF0004CF20003C4F20F034FF00002C3F8A82103
:103000004CF20003C4F20F034FF00002C3F8AC21EE
:103010004CF20003C4F20F034FF00102C3F80C217D
:103020004CF20003C4F20F0340F26302C0F2050247
:10303000C3F884204CF20003C4F20F034FF0AA023D
:10304000C3F88C204CF20003C4F20F034FF055027A
:10305000C3F88C204CF20003C4F20F034FF00102BE
:10306000C3F880204CF20003C4F20F034FF0AA0211
:10307000C3F88C204CF20003C4F20F034FF055024A
:10308000C3F88C204CF20003C4F20F03D3F888304D
:1030900003F08063002BF5D04CF20003C4F20F0361
:1030A0004FF00302C3F880204CF20003C4F20F0378
:1030B0004FF0AA02C3F88C204CF20003C4F20F03B5
:1030C0004FF05502C3F88C204CF20003C4F20F03FA
:1030D000D3F8883003F04073002BF5D04CF2000396
:1030E000C4F20F034FF02302C3F8A4204CF20003F4
:1030F000C4F20F034FF0AA02C3F8AC204CF2000355
:10310000C4F20F034FF05502C3F8AC204CF2000399
:10311000C4F20F034FF00102C3F8A0204CF20003E9
:10312000C4F20F034FF0AA02C3F8AC204CF2000324
:10313000C4F20F034FF05502C3F8AC204CF2000369
:10314000C4F20F03D3F8A83003F48063002BF5D04A
:103150004CF20003C4F20F034FF00302C3F8A020A7
:103160004CF20003C4F20F034FF0AA02C3F8AC20E4
:103170004CF20003C4F20F034FF05502C3F8AC2029
:103180004CF20003C4F20F03D3F8A83003F44073E9
:10319000002BF5D04CF20003C4F20F0348F2DE72AC
:1031A000C0F22842C3F8C4204CF20003C4F20F035B
:1031B0004FF00002C3F8C8214CF20003C4F20F0321
:1031C00043F23A021A604EF60053CEF200034FF07B
:1031D00000029A60704700BF08B500F04BF807483E
:1031E00000B10068064901B109680022FDF702F844
:1031F000044B0BB1AFF30080FEE700BF00000000FE
:10320000000000000000000080B51448144B21E0CD
:103210005C689968DD688C420CD0002205E0A61835
:103220000832D6E9008941E902898C460831AA4270
:10323000F5D101E004EB050C1C696146002204E0B5
:1032400008320026002741E902670831A242F7D17F
:10325000143301380028DBD1FFF7BEFF0100000066
:10326000E433000001498D46014908470080001001
:103270000932000070B543F2D03643F2D035C0F2C7
:103280000006C0F20005761BB61006D0002455F8E3
:10329000243001349847A642F9D843F2D03543F29E
:1032A000D436C0F20005C0F20006761B00F08AF8A2
:1032B000B61006D0002455F8243001349847A642B1
:1032C000F9D870BD1201000202000008C91F0220D7
:1032D0000001010203010000090243000201008015
:1032E0003209040000010202005E052400100105FD
:1032F00024010101042402020524060001070581BE
:103300000310000209040100020A00005E07050222
:103310000240000007058202400000000403090487
:103320001C034E00580050002000530045004D0083
:10333000490043004F004E004400200024034E008B
:103340005800500020004C0050004300310037006E
:10335000780078002000560043004F004D00200008
:103360001A03440045004D004F003000300030008B
:10337000300030003000300030000A0356004300B7
:103380004F004D00191E0000A92C0000E92C000080
:10339000000000000000000000000000000000002D
:1033A000000000000000000000000000000000001D
:1033B000000000000000000000000000000000000D
:1033C00000000000F8B500BFF8BC08BC9E4670477E
:1033D000F1000000F8B500BFF8BC08BC9E4670477D
:1033E000DD000000000000000034000000000010BC
:0833F00018000000900200002B
:0833F800D4CCFF7F01000000AE
:10340000000000000000000000C2010000000800F1
:083410000100000000E1F505D8
:00000001FF
